:100000000C9450030C9488030C9488030C94922B4A
:100010000C9488030C9488030C9488030C94880334
:100020000C9488030C9488030C94CF290C94A72A71
:100030000C9484290C9488030C9488030C948803F2
:100040000C9488030C9488030C9488030C94880304
:100050000C9488030C94AB290C9488030C948803AB
:100060000C9488030C9488030C9488030C948803E4
:100070000C9488030C9488030C9488030C948803D4
:100080000C9488030C9488030C9488030C948803C4
:100090000C9488030C9488030C9488030C948803B4
:1000A0000C9488030C9488030C94880305010902BE
:1000B000A10185020901A1000509190129081500FE
:1000C0002501950875018102050109300931158165
:1000D000257F95027508810609381581257F9501D0
:1000E00075088106050C0A38021581257F95017572
:1000F000088106C0C005010980A101850319012AF4
:10010000B700150126B700950175108100C0050CD8
:100110000901A101850419012AA002150126A002E6
:10012000950175108100C005010906A10105071997
:10013000E029E715002501950875018102950175F3
:100140000881010507190029FF150026FF00950603
:1001500075088100050819012905950575019102A9
:10016000950175039101C009023B00020100A0FA4C
:10017000090400000103010100092111010001220D
:100180004000070581030800010904010001030084
:100190000000092111010001227B000705820320D4
:1001A000000112010002000000081D8D3A34000118
:1001B0000102000124034100750072006F0072000B
:1001C0006100200043006F0072006E006500200097
:1001D00072006500760031000000180373007000A3
:1001E0006C00690074006B0062002E0063006F00F9
:1001F0006D0000000403090400000000000000007E
:1002000000000000000000000000000000000000EE
:100210000000000000000000000000007E0F00D47D
:10022000FFFFFFC700000078000000000000000092
:100230002A2B280000000000000000000000000041
:1002400000000029000000002C1E3420212224344C
:100250002627252E362D3738271E1F20212223241E
:1002600025263333362E37381F0405060708090ABA
:100270000B0C0D0E0F101112131415161718191A56
:100280001B1C1D2F3130232D350405060708090AD4
:100290000B0C0D0E0F101112131415161718191A36
:1002A0001B1C1D2F3130354C2223252628292A2CB2
:1002B0002D2F3032333536383A3B3D3E40424345B0
:1002C00047494A4C4E5051535557595A5C5E6062EB
:1002D000646668696B6D6F71737577797B7D7F81FB
:1002E000838587898A8C8E90929496989A9C9E9FFB
:1002F000A1A3A5A7A8AAACAEAFB1B3B4B6B8B9BB19
:10030000BCBEBFC1C2C3C5C6C7C9CACBCCCDCED087
:10031000D1D2D2D3D4D5D6D7D7D8D9D9DADADBDB74
:10032000DBDCDCDCDCDCDDDDDDDDDCDCDCDCDCDB0B
:10033000DBDBDADAD9D9D8D7D7D6D5D4D3D2D2D154
:10034000D0CECDCCCBCAC9C7C6C5C3C2C1BFBEBC47
:10035000BBB9B8B6B4B3B1AFAEACAAA8A7A5A3A1B8
:100360009F9E9C9A98969492908E8C8A898785837A
:10037000817F7D7B79777573716F6D6B696866645A
:1003800062605E5C5A5957555351504E4C4A49472A
:10039000454342403E3D3B3A3836353332302F2DCF
:1003A0002C2A292826252322FFAA7F554000010157
:1003B0000101010101010102020202020202020224
:1003C00003030303030303030404040404040405F4
:1003D00005050505060606060607070707070808B8
:1003E0000808090909090A0A0A0B0B0B0C0C0C0D69
:1003F0000D0D0E0E0E0F0F0F101011111112121302
:10040000131414151516161717181819191A1A1B7C
:100410001B1C1D1D1E1E1F202021222223242425DB
:100420002626272829292A2B2C2D2D2E2F30313214
:1004300032333435363738393A3B3C3D3E3F404124
:1004400042434445464748494A4C4D4E4F5051530C
:1004500054555658595A5B5D5E5F616264656668C3
:10046000696B6C6D6F7072737577787A7B7D7E8047
:1004700082838587888A8C8E8F91939596989A9C93
:100480009EA0A2A3A5A7A9ABADAFB1B3B5B7BABCA7
:10049000BEC0C2C4C6C9CBCDCFD1D4D6D8DBDDDF78
:1004A000E2E4E7E9EBEEF0F3F5F8FAFDFF1E0F05E5
:1004B0007F3F1F643214643214783C1E1E140A05F8
:1004C0002B4414001A000900130005002921040020
:1004D0001500160017000A001A7C1D001B000600FC
:1004E0000700190000000000000081522C004C2879
:1004F0002A2433001C0018000F000D0034311200B4
:100500000C000800110010001B7C3800370036007A
:100510000B000E00000000000000025228432C34A3
:100520002B441E021F0220022102220229212252F4
:100530000000000027000000E100000000000000B3
:1005400000000000000000000000015200522A28B4
:100550002A24270226022502240223023500310024
:1005600030002F002E002D003502310230022F0204
:100570002E022D02000000000000035228432C34FC
:100580002B443A003B003C003D003E0029213F0047
:1005900040004100420043001A7C000000000000BF
:1005A00044004500000000000000045200522A28C8
:1005B0002A24270026002500240023022E002D00D7
:1005C00023002200210036002502380020001F00F1
:1005D0001E003700000000000000035228432C34A6
:1005E000A800AC00AB00AA00A900AE0029210000C1
:1005F0000000D300D100D200E100000000000000A4
:100600000000000000000000000004520052E3005F
:10061000DD0000000000DC00D000CE00DE000000A5
:100620000000DA00D9000000DF0000000000DB005D
:10063000CF00CD000000000000000000000000001E
:1006400020782C782B7828782778307846002D78F9
:100650002E78247823783478E10032782F78267841
:100660002578317800000000000000000052E3000F
:10067000005200004A004B004F00510000000000F3
:100680000000000000000000000000004D004E00CF
:100690005000520000000000000003522800E30058
:1006A00011241FBECFEFDAE0DEBFCDBF04B603FEDC
:1006B00018C08091BD049091BE04A091BF04B09178
:1006C000C0048730904BA740B04B59F41092BD0442
:1006D0001092BE041092BF041092C004E0E0F8E350
:1006E000099524E0ACEDB1E001C01D92AD3BB2072D
:1006F000E1F711E0A0E0B1E0E0E7FEE502C005901F
:100700000D92AC3DB107D9F70E9427240C94C72E57
:100710000C9400009C01FB019A9581159F4130F4D7
:10072000832F817031FD82600995089580E0FCCFB0
:100730009093710480937004089590937304809350
:100740007204089521E030E002C0220F331F8A9521
:10075000E2F78091720490917304822B932B0E9494
:100760009D03089521E030E002C0220F331F8A95D7
:10077000E2F7209530958091720490917304822362
:1007800093230E949D030895983098F5863088F54C
:10079000E82FF0E086E0989FE00DF11D11248E2FE8
:1007A000877041E001C0440F8A95EAF783E0F6952F
:1007B000E7958A95E1F7EE0FFF1FEE0FFF1FEB5C49
:1007C000FB4F20E030E070E05191DF011197CB0149
:1007D000022E02C0969587950A94E2F78170819562
:1007E0008527842385278C932F5F3F4F2430310545
:1007F00059F70895983078F5863068F5E82FF0E0DD
:1008000086E0989FE00DF11D11249E2F977083E0E4
:10081000F695E7958A95E1F7EE0FFF1FEE0FFF1FA4
:10082000EB5CFB4F40E050E080E0219130E0092E8E
:1008300002C0369527950A94E2F721703327042EDB
:1008400001C0220F0A94EAF7822B4F5F5F4F4430BA
:10085000510559F7089580E0089580917B049091A7
:100860007A04981301C008958F5F8770FACFE0EE85
:10087000F1E09191891303C0DF0111971C9291E07F
:10088000E63EF907B1F708959091750480958923A4
:1008900080937504282F2770211111C0891779F0D2
:1008A0009091BC0492FF0BC08695869586950E9418
:1008B000B203109275041092770410927604089592
:1008C000982F909580916E04892380936E040895EB
:1008D00080916D04811531F010926D0410927904AD
:1008E0001092780408957830B8F46630A8F4853012
:1008F000B0F4E62FF0E096E0799FE00DF11D1124B1
:1009000090E3899FE00DF11D1124EE0FFF1FE054CD
:10091000FB4F85919491089580E090E0089581E0E7
:10092000FCCF803E9105D9F1C8F48133910509F4DB
:1009300082C048F48932910509F472C08A32910567
:1009400009F480C0089589339105E9F08238910552
:10095000D1F08533910509F45EC00895843E910578
:10096000D9F148F4823E910539F1833E910549F170
:1009700081EE90E00895863E9105C9F1873E91058C
:1009800009F43EC008952091BB042370211164C076
:100990002091BC0423FF14C089E290E008952091C7
:1009A000BB0420FD45C03091BC0430FF09C024FDCC
:1009B00024C083EE90E008952091BB0422FDF7CF80
:1009C00008952091BB0422FD44C03091BC0430FD49
:1009D00043C024FFF5CF11C02091BC0421FFF0CF0C
:1009E0008091BB0484FD09C087EE90E008952091BA
:1009F000BB0423FFE5CF24FFF7CF80E090E008950C
:100A00002091BB0423FD2BC03091BC0431FFE1CF0A
:100A100084EE90E008952091BB0425FFD1CFBCCF98
:100A20002091BB0425FD1EC02091BC0423FFC8CF2C
:100A300089E390E008952091BB0426FFC1CF8AE2AC
:100A400090E008952091BB0426FFBACF81E390E0A7
:100A5000089582EE90E0089580EE90E0089586EE8D
:100A600090E0089585E390E008959091BB0492FF93
:100A700006C0282F28712830F9F4877F846093FFFF
:100A800006C0282F28712831F1F4877E84612091D7
:100A9000BC0420FF06C0382F38713830D9F4877F66
:100AA000816021FF06C0282F28712831D1F4877E6C
:100AB000816194FD877E0895282F24712430F9F6F2
:100AC0008B7F8860DCCF282F2471243101F78B7E47
:100AD0008861DDCF382F3171313019F78E7F886012
:100AE000E0CF282F2171213121F78E7E8861E1CF5F
:100AF0001F93CF93DF930E949104EC01811522E5AF
:100B0000920708F05DC0811540E5940708F0DBC04E
:100B1000803E910528F58D3C910508F0ACC0883ADF
:100B2000910578F4853A910508F0A2C081309105CD
:100B300009F441C00497813A9105E8F1C0E0D0E0A2
:100B40003AC0885A91094B97C8F7C85AD0E0CC0FE1
:100B5000DD1FCA55DE4F0990D881C02DD4642BC04B
:100B6000811550E49507F8F4C11580E2D80708F024
:100B7000C3C0C83ED105F8F0CE019A9581159F41BA
:100B8000E8F68D2F0E943505182FCE0199270E9477
:100B90009104212F30E0322F2227E901CC27DF7189
:100BA000C82BD92B08C099270E949104CC27DF704D
:100BB000C82BD92BD06ACE01DF91CF911F91089518
:100BC000803842E59407C8F5803652E5950708F06D
:100BD0005BC0C03482E5D807D0F4C03292E5D907B3
:100BE00008F04BC08C2F8695869520E2829FC0012D
:100BF0001124C37021E030E0A90102C0440F551F49
:100C0000CA95E2F7EA01C82BD92BDD68D4CF8C2F27
:100C100086958695877050E2859FC0011124C37028
:100C200021E030E0A90102C0440F551FCA95E2F748
:100C3000EA01C82BD92BDC68BECF803C52E5950772
:100C400058F48F71C03AD245A0F590E0982F8827CC
:100C5000EC01C46FD06AAFCF805C9245809708F0FA
:100C60006DCFDC2FCC27CC27DF71C06FD06AA3CF2C
:100C7000A497D064A0CFD0659ECFCF71D0E0DC2FF9
:100C8000CC27C16FD06A97CF86958695877020E272
:100C9000829FC0011124C37021E030E0A90102C08D
:100CA000440F551FCA95E2F7EA01C82BD92BDA6821
:100CB00082CF0E943505C82FD0E0DC2FCC27CC276F
:100CC000DF71D06278CF8F710E94350565E0D695CF
:100CD000C7956A95E1F7CF70D0E0DC2FCC27282F9D
:100CE00030E084FF05C054E0220F331F5A95E1F72E
:100CF000C22BD32BD0695FCF8D2F8F710E9435050A
:100D0000182FCE0199270E949104212F30E0322F15
:100D1000222722273F71282B392BE901D2CFA0E0CF
:100D2000B0E0E5E9F6E00C94B62C8C01E09072049A
:100D3000F09073048091700490917104E82AF92A6C
:100D4000CFE0D0E0CC24C394D12CC6010C2E02C03D
:100D5000880F991F0A94E2F78E219F21892B49F46D
:100D6000219798F7B12C8B2DCDB7DEB7E9E00C9425
:100D7000D22CBC2EB8018C2F0E9473040E947805DF
:100D8000019771F3F0CF0F931F93CF93FC018581EF
:100D900000811181811591F0611581F0C8010E94D7
:100DA0008F06C82F682FC8010E94C403B8018C2F7A
:100DB0000E947304CF911F910F910895C8010E9462
:100DC000FA03C82FF3CFCF93DF93D82FC92F0E94F8
:100DD0008F066D2F7C2F0E9473040E947805DF918F
:100DE000CF910895FC0184818115A1F080819181CA
:100DF0000E94E306282F92959F70963099F060F438
:100E0000925F9F70923030F4203F89F038F481E097
:100E1000283E38F080E008959A5FF3CF81E0243FC8
:100E2000C9F7089581E0283E20F0213FF9CF81E005
:100E30000895089580E00895F894E82FE295EF7002
:100E4000F0E041A18F7021E030E0B90102C0660FEF
:100E5000771F8A95E2F7CB01962F9095942391A363
:100E600092A1892B82A378940895089580914F04CC
:100E700080FD14C081FD14C082FD16C080914E0417
:100E8000811581F08E3180F420E5829FC00111240C
:100E90006EE170E00E94122D862F089584E108957E
:100EA00088E2089588E0089580E5089580914F04D0
:100EB00080FD17C081FD17C082FD19C080914D04CF
:100EC000811599F0883298F428E0829FC00111249E
:100ED00068E270E00E94122D6115710551F0862FB5
:100EE000089562E0FCCF64E0FACF61E0F8CF68E0FB
:100EF000F6CF81E00895A0E0B0E0E1E8F7E00C94DF
:100F0000B62C8901E42FF0E0E355FC4F61110FC0CE
:100F1000E491BE2E2E2FD80111962C931197EC93AD
:100F20001296BC92CDB7DEB7E9E00C94D22CC82F54
:100F3000D0E0E62EF12C3491232F86E08C9F6001C7
:100F40008D9FD00C1124EFEFF0E0C601BF010E948D
:100F5000FE2CCC0FDD1F45E5469FC001479F900D3D
:100F60001124C81BD90BAC2FAA0FAC0FAF014E191F
:100F70005F09349FC001359F900D1124B92EAE9D9D
:100F8000E001AF9DD00D1124CD2FDD27AF014C1B0B
:100F90005D0BEA013C9FA0013D9F500D1124EF0124
:100FA000CA1BD109DE01AE9DE001AF9DD00DBE9DF3
:100FB000D00D1124CD2FDD27EC1BFD0B3E9FD00162
:100FC0003F9FB00D1124EB2F63307105D1F0DCEFA2
:100FD000CD16D3E0DD0658F461307105B1F0623012
:100FE000710509F098CFE32F292FBB2E94CF6430E1
:100FF000710571F06630710509F48DCFE92FB52EBA
:101000008ACF292FB32EE52F86CFE32F252F83CF2D
:10101000E92FB32E2B2F7FCF80916504823060F4AF
:10102000817082608093650480916804813818F033
:1010300080E88093680408958235B0F381708065FC
:10104000F1CFE2E6F4E01182828184608283089528
:10105000FA01811511F009950895FB01FCCFFC01FF
:10106000680F791F8FEF41E39191892728E030E0E5
:10107000982F990F87FF09C0892F8427215030406E
:10108000B9F7E617F70781F70895892FF7CFA3E09F
:10109000B0E0EDE4F8E00C94BD2C9C0180910A02D4
:1010A00090910B0282179307A1F030930B022093CB
:1010B0000A02E0912B04F0912C04309751F083E068
:1010C00089833B832A830680F781E02DCE01019638
:1010D00009952396E2E00C94D92CA3E0B0E0E3E775
:1010E000F8E00C94BD2C9C018091080290910902BB
:1010F00082179307A1F03093090220930802E09130
:101100002B04F0912C04309751F084E089833B83C9
:101110002A830680F781E02DCE010196099523965A
:10112000E2E00C94D92C9C01FC0132968FEF90E008
:101130004191461751F08F3F19F4411101C0892F99
:101140009F5F9630A9F78F3F09F40895280F311D4E
:1011500087FD3A95F901628308952FB7F89480913D
:10116000090490910A04A0910B04B0910C042FBFC4
:101170000895962F2091BC0422FF10C0682F660F9F
:10118000660F660F692B609375040E94A2030E948C
:10119000AD08909377048093760408950E94A2038B
:1011A000089590916D04292F2823211561F08095D1
:1011B000892380936D04811539F00E94AD088093D6
:1011C000780490937904089580E090E0F8CF0E942D
:1011D000AD082091520430915304232B211521F0A6
:1011E0008093EE039093EF032091540430915504C3
:1011F000232B211521F08093EC039093ED03E091D4
:101200002B04F0912C04309749F082E08093500435
:101210000480F581E02D80E594E00995089561153D
:1012200009F44BC0E3E3E80FE33150F4F0E0E75397
:10123000F14D0C94262D0E9436078195809353041E
:101240000E94E70808950E943607F8CF0E943607EB
:10125000819580935204F4CF0E943607FACF0E9402
:10126000560780935404ECCF0E9456078195F9CF1E
:101270000E945607819580935504E2CF0E9456073D
:10128000FACF815D990B21E030E001C0220F8A95F1
:10129000EAF780915104822B80935104D1CF809141
:1012A0004F04816080934F04CBCF80914F048260C4
:1012B000F9CF80914F048460F5CF409152048D3C6A
:1012C00059F48091530487FF0DC0109253044115C7
:1012D00059F410924E0408C08E3C81F4809153045E
:1012E00018169CF3411581F0809154049091550497
:1012F000892B8111A5CF10924D04A2CF8F3C41F4D0
:1013000047FFF0CF10925204809153048115E0CF33
:10131000803D19F41416B4F3E5CF90915404893D3F
:1013200029F41916FCF610925404DCCF8A3D19F406
:1013300097FFD8CFF8CF909155048B3D29F497FFB4
:10134000D1CF10925504CECF8C3D19F41916CCF3A1
:10135000C9CF9FE2980F983090F4815D990B21E0FE
:1013600030E0B90102C0660F771F8A95E2F7CB0122
:10137000809590915104892380935104B3CF8D3D82
:1013800031F480914F048E7F80934F04ABCF8E3D1C
:1013900021F480914F048D7FF7CF8F3D09F0A2CFCC
:1013A00080914F048B7FF0CF2FB7F89460910904A0
:1013B00070910A0480910B0490910C042FBF089542
:1013C0009C014FB7F8948091090490910A04A09170
:1013D0000B04B0910C044FBF821B930B08958091B6
:1013E00007020895FC019B018091FD019091FE018F
:1013F0008617970740F0672B29F48091E8008E77D5
:101400008093E800C90140E0009741F4411106C013
:101410008091E80082FF2FC080E00895209123048E
:101420002115A9F12530A9F12091E80023FD2DC057
:101430002091E80022FDECCF2091E80020FFE4CFCE
:101440003091F3002091F200009719F02830310517
:1014500058F041E02830310509F040E02091E800E3
:101460002E772093E800D0CF41914093F10001976F
:101470002F5F3F4FE9CF80912304811541F08530E4
:1014800041F08091E80083FFC3CF81E0089582E0BE
:10149000089583E008958091F70187FF13C080913C
:1014A000E80082FF06C08091E8008B778093E80017
:1014B0000895809123048111F2CF0895809123042F
:1014C0008115D9F38091E80080FFF8CF8091E80082
:1014D0008E77ECCF2091E4003091E50095E6A901EC
:1014E0008091EC008170811531F08091E80080FFDF
:1014F00006C080E008952091E80022FD1AC0809186
:101500002304811589F0853089F08091EB0085FDF9
:101510000FC02091E4003091E5004217530701F31A
:101520009A95E9F684E0089582E0089583E00895AD
:1015300081E00895E8EDF0E080818E7F8083109255
:10154000E2001092DA001092E100A0EEB0E08C917F
:1015500081608C9380818F77808319BCA7EDB0E088
:101560008C918E7F8C9380818F7E80831092F60188
:101570000895982F9093E900242F762F50E0981724
:1015800031F07091EC002091ED005091F00021FDC0
:1015900006C09F5F973071F78093E90008953091FE
:1015A000EB003E7F3093EB003091ED003D7F3093B8
:1015B000ED003091EB0031603093EB007093EC0064
:1015C0002093ED005093F0002091EE0027FDE1CF35
:1015D0000895A0E0B0E0EFEEFAE00C94B72CC8ED6F
:1015E000D0E088818F7E8883E7EDF0E080818160A4
:1015F000808384E082BF81E08093F60188818E7FC2
:10160000888302EE10E0F80110821092DA0081EE79
:10161000C82ED12CF601108288818F77888388812B
:101620008068888388818F7D888319BC1092230409
:101630001092F5011092CB031092F40190EEE92E76
:10164000F12CF70180818B7F808388818160888382
:1016500042E060E080E00E94B90AF60180818E7F5E
:101660008083F801808181608083808188608083AD
:10167000F70180818E7F8083888180618883CDB7E8
:10168000DEB7E8E00C94D32CE0917B0490917A04CF
:1016900027E0E91302C080E00895AE2FB0E02E9F4E
:1016A000F0011124E458FB4F3181361306C030811C
:1016B000381303C03581341304C0FD013196E7703F
:1016C000E8CF81E0089580912404811110C08091B9
:1016D000D80080618093D8008AE18A95F1F700C034
:1016E0008091D90080FF0AC081E08093240481E0CA
:1016F00090912404913009F080E0089582E0809375
:1017000024040E949A0A10922304F1CF0F931F938E
:101710000E94630B811529F00E94D4091F910F913B
:1017200008950E94D4090091250410912604209167
:10173000270430912804600F711F821F931FEECF82
:101740000E94860B08950E94630B811519F00E9478
:10175000AD0808950E94860BCB0108950E94630B8B
:10176000811559F0E0912B04F0912C04309729F069
:101770000190F081E02D0995089580E00895409151
:1017800014018091650480FF24C02091130130E092
:10179000C901880F991F820F931F845E9C4F539A33
:1017A0006BB1677F7BB17860EFB7F89450E09A0136
:1017B000220F331F240F351F280F391F2817390711
:1017C000E9F4EFBF8FE594E00197F1F700C0000066
:1017D00008958091150190911601282F30E0F901AC
:1017E000EE0FFF1FE20FF31FE45EFC4F891768F650
:1017F0001182108212828F5F3396F8CFDC014D91F7
:10180000CD0158E07BB9000000C047FF6BB9440F21
:10181000000000C000C000C06BB900C05A9591F72D
:10182000CDCFEF92FF921F93CF93DF93EC0110E0A7
:10183000EE24EA94F12C60911701161770F00E94C3
:10184000BF0B9A818C8190FF28C08F5F8C83DF91C2
:10185000CF911F91FF90EF90089580911501810F16
:101860009927991F9C01220F331F280F391F245ECF
:101870003C4F40916804413808F040E870E0C701EF
:101880000E94122D962F8C8160916704199F800D04
:1018900011240E947B071F5FCECF8150D7CFA0E0DD
:1018A000B0E0E5E5FCE00C94B42CEC018A81BB24AB
:1018B000B39480FF02C0BB24BA948C81A09017011E
:1018C000811109C091E0B91202C08FEF8A0D809397
:1018D0001B0381E08C83E12CF12CEA14B8F00E9408
:1018E000BF0B90911B03E1E0BE1255C08091170120
:1018F0008150911519F08FEF890F91E080931B03B0
:101900009C83CDB7DEB7EBE00C94D02C8091150111
:101910008E0D9F2D911D8C01000F111F080F191F97
:10192000045E1C4FF80111821082128234E0C32E33
:10193000D12C912C80911B03890D873344F166E3F0
:101940000E94F02C892F082E001C00088E150F0411
:10195000A9F4809168048C9DA0018D9D500D1124E7
:101960005595479555954795413808F040E89801B9
:1019700060916704809166040E947B079B0CF1E0F4
:10198000CF1AD108B9F68FEFE81AF80AA6CF87FF69
:10199000DACF8A0DD8CF892F90E001966091170198
:1019A00070E00E94122D982FA9CF0F931F93CF9311
:1019B000DF93EC018C81811109C081E08C8310924E
:1019C0001A0392E09093070180930601109115018C
:1019D00020911601812F90E0FC01EE0FFF1FE80F10
:1019E000F91FE45EFC4F821750F100E0609117018F
:1019F000061758F10E94BF0B8091060190911A03BF
:101A0000980F90931A0320910701280F2093070144
:101A1000121654F4209117012150330B092E001C8B
:101A200000089217030634F08195809306018130F7
:101A300009F41C82DF91CF911F910F9108951182BB
:101A4000108212828F5F3396CECF202F30E070E06D
:101A5000C9010E94122D810F90E040911A03FC01F0
:101A6000EE0FFF1FE80FF91F042E001C00082417BB
:101A70003005C4F040910701042E001C00084217F5
:101A8000030684F09F01245E3C4F40916804413876
:101A900008F040E860916704809166040E947B072B
:101AA0000F5FA4CFE45EFC4F118210821282F8CF48
:101AB000A6E0B0E0EEE5FDE00C94B72C8D839E83AC
:101AC000AD81BE811496FC912F2F30E0D9010E9488
:101AD000B82E9B01AC010E94832E6B017C0180E239
:101AE00090E09C012F1B3109F901A5E5B0E0A701A9
:101AF00096010E94832E69837A838B839C839F0146
:101B0000DF010E942C2D9B01AC010E948E2E9B01B7
:101B1000AC012C0D3D1D4E1D5F1D69817A818B81AD
:101B20009C810E94962E022F30E00A3248F5C901AE
:101B3000880F991F820F931F95958795F82EF09423
:101B400010E085E5E82EE01A80911701181738F1AA
:101B50000E94BF0BAD81BE8114969C9181E09115CE
:101B600019F0903219F48FEF8093050180910501EF
:101B7000890FED81FE8184832696E8E00C94D32CB6
:101B800085E590E0AC01421B530B9A01CA01880F16
:101B9000991F820F931F97FFCFCF0196CDCF8E2D28
:101BA00011FD802F40911501410F5527551F9A01B6
:101BB000220F331F240F351F245E3C4F4F2D51E859
:101BC000F51608F040E8609167040E947B071F5FEC
:101BD000BBCF9091650490FF11C090911501509179
:101BE0001601292F30E0F901EE0FFF1FE20FF31F5E
:101BF000E45EFC4F951718F00E94BF0B0895818397
:101C0000608342839F5F3396F5CFA3E0B0E0EBE0C3
:101C1000FEE00C94BD2C9091650490FF0DC04138FE
:101C200008F040E89E012F5F3F4F0E947B074B81E9
:101C300069818A810E94E90D2396E2E00C94D92CF7
:101C4000CF93DF93EC01EC81F0E0E855FD4F449138
:101C5000E5E6F4E0628181810E94050E8C818F5F50
:101C60008C83DF91CF910895CF93DF93EC01E5E66C
:101C7000F4E0438162818C810E94050E8C818F5F2C
:101C80008C83DF91CF91089581E08093E00080E222
:101C90008093D8001092C9008FE19EE40197F1F77C
:101CA00000C0000087E090EBDC018093BD049093BE
:101CB000BE04A093BF04B093C00488E19CE00FB6BB
:101CC000F894A895809360000FBE90936000FFCFBA
:101CD0000F931F93CF93DF938B01EA01909123041D
:101CE000943059F58093E9008FEF9091E80095FDCD
:101CF00006C095ED9A95F1F700008A95B1F78091AD
:101D0000E80085FF1AC00E946A0A811111C0809103
:101D1000E80085FD06C08091E8008E778093E8009A
:101D2000F2CFF80181918F018093F100219779F72B
:101D30008091E8008E778093E800DF91CF911F912A
:101D40000F910895CF93DF93D82FC92F48E050E02B
:101D5000682F792F81E00E94680E88E0ED2FFC2F1C
:101D6000AFEFB1E001900D928A95E1F7DF91CF914D
:101D70000895BC0146E050E082E00E94680E08959C
:101D8000BC0143E050E082E00E94680E0895A0E0AC
:101D9000B0E0EDECFEE00C94B52CF82EE92EB62E5A
:101DA000A72E8A018091F001CC24C394D12C8A30D3
:101DB00018F48AE0C82ED12CC1E0D0E06B2D7A2D2A
:101DC0008F2D9E2DF8010995811116C02196CC16F4
:101DD000DD0694F0CC9FC001CD9F900D900D112495
:101DE00020E030E045E34A95F1F700002F5F3F4FD8
:101DF00028173907B9F7E2CFCDB7DEB7EAE00C9480
:101E0000D12C9091BC0492FB222720F9281779F05D
:101E100080FB92F99093BC046091BB047091BC0468
:101E200084E090E00E944E2E82E00E9444040895D7
:101E3000609158048CE090E00E94302E089520912B
:101E4000C803082E000C990B820F911D27FD9A954F
:101E500063E070E00E94122DE82F87FF02C0E3E0EC
:101E6000E80FE093C8030E2E000CFF0BEF56FE4F59
:101E70008081809358040E94180F089580916E0409
:101E800090917404892B8093DE0180916D048115FB
:101E900019F10E94AD082091780430917904821BD9
:101EA000930B8838934110F00E9468048091DE0102
:101EB00090916D04892B8093DE0120E080EE91E00B
:101EC000FC013081019631112F5F31E0863E93078E
:101ED000B9F721110E94680448E050E06DE274E017
:101EE0008EED91E00E94F62D892BA9F088E0EEEDB1
:101EF000F1E0ADE2B4E001900D928A95E1F7E09156
:101F00002B04F0912C04309731F00280F381E02D06
:101F10008EED91E009950895811521F00E946004ED
:101F20000E943E0F0895811541F0809590917404B0
:101F30008923809374040E943E0F0895811539F01F
:101F400090916E04892B80936E040E943E0F089539
:101F5000811539F090917404892B809374040E9448
:101F60003E0F0895CF93C82F8115A9F08CEF8C0FE9
:101F7000813A98F4E0EEF1E08191C81709F440C08D
:101F800021E0E63EF207C1F76C2F8EED91E00E9452
:101F900093080E943E0FCF91089580E28C0F883005
:101FA00068F4C77021E030E001C0220FCA95EAF75B
:101FB00080916E04822B80936E04EBCF8BE58C0FA7
:101FC000833038F42C2F2452330BC9010E94470868
:101FD000E2CFE8E5EC0FEB3150F4F0E0EE0FFF1F3D
:101FE000EA55FE4F808191810E946D08D4CF83E332
:101FF0008C0F833180F661E08C2F0E940F09CBCFCC
:102000008C2F0E9437040E943E0FBECF811581F1B4
:102010009CEF980F913A28F40E9437040E943E0FDB
:10202000089590E2980F983050F4877091E001C0C5
:10203000990F8A95EAF7892F0E946004EFCF9BE5FC
:10204000980F933028F480E090E00E9447080895AC
:1020500098E5980F9B3128F480E090E00E946D088D
:10206000089593E3980F933118F460E00E940F09EC
:102070000895EF92FF920F931F93CF93DF93EC019C
:102080008B017C0180EEE81AF1086EE97FE098E0B0
:10209000E916F10410F068EA7FE0CE010E948A039D
:1020A0008C2F0E94B20F0115110599F48C2F0E94FC
:1020B00006106CE87FE098E0E916F10410F063E99F
:1020C0007FE0CE010E948A03CDB7DEB7E6E00C9434
:1020D000D52C8FE99FE00197F1F700C00000015077
:1020E0001109E1CF0F931F93CF93C82F00E510E0A4
:1020F000893311F000E010E08C2F0E94B20F01151F
:10210000110539F48C2F0E940610CF911F910F9169
:1021100008958FE99FE00197F1F700C0000001509A
:102120001109EDCFFF920F931F93CF93DF93C62F2B
:10213000D42F122F8115A9F0609360040E94AD087E
:102140009093F2018093F101C77081E001C0880F84
:10215000CA95EAF70E949E0FCDB7DEB7E5E00C9472
:10216000D62C80916004681334C08091F101909165
:10217000F2010E94E00920915F0130916001821715
:10218000930738F500E20D0FCD17A9F0C770FF24B3
:10219000F3948F2D01C0880FCA95EAF70E948C0F27
:1021A000083048F48D2F877001C0FF0C8A95EAF73C
:1021B0008F2D0E949E0F812F0E947210083060F6B2
:1021C000D77081E001C0880FDA95EAF70E948C0F82
:1021D000C3CFC77081E001C0880FCA95EAF7F6CF78
:1021E000811107C089EA611101C08AEA0E94721058
:1021F00008958130E9F78EE46111F8CF8BE4F6CFD2
:10220000A0E0B0E0E6E0F1E10C94B82CE82FF0E0BB
:10221000E85DFD4FD490282F26952695269530E031
:10222000F901E85EFD4F0491877010E0082E02C0AE
:10223000159507950A94E2F701701127F901E85FF7
:10224000FD4FE490F12C082E02C0F594E7940A9417
:10225000E2F791E0E922FF24F901E850FE4FC49132
:10226000D0E002C0D595C7958A95E2F7C170DD2709
:102270000115110519F081EE0E94B20FE114F1046D
:1022800019F086EE0E94B20F8D2D0E947210E1149B
:10229000F10419F086EE0E9406100115110519F0DF
:1022A00081EE0E940610CD2B19F08CE20E94721074
:1022B000CDB7DEB7E7E00C94D42CCF9310926E0428
:1022C000C6E0E0EEF1E0DF018C2F1D928A95E9F780
:1022D00080E090E00E94470880E090E00E946D0856
:1022E000109274040E943E0FE0E5F4E0DF011D92BD
:1022F000CA95E9F710924E0410924D0410924F04C3
:102300000E94E708CF9108950E945D112FEF84E3AA
:102310009CE0215080409040E1F700C0000088E13F
:102320009CE00FB6F894A895809360000FBE909340
:102330006000FFCFAAE2B0E0E0EAF1E10C94BC2C2F
:1023400087EF91E0FC0101962091F100208321E0CC
:102350008F3F9207B9F78091F801893009F456C090
:10236000C8F4823009F4B2C0833009F481C08130EE
:1023700071F18091E80083FFE7C08091F7019091AF
:10238000F8019A3008F0E0C0E92FF0E0E452F14D96
:102390000C94262D8A3009F488C08B3051F7809137
:1023A000F701813231F78091FB019091FC01892B7B
:1023B00001F78091E800877F8093E8000E944B0A34
:1023C0008091F901809304010E945D11D2CF809128
:1023D000F701813A71F68091E800877F8093E800E9
:1023E0008091FB019091FC01892B61F060E080E01D
:1023F00090E070E00E94F2098091E8008B77809372
:10240000E800B7CF68E08FEF91E0F3CF8091F7015C
:10241000813209F0AECF8091FB019091FC010297CF
:1024200008F0A7CF8091E800877F8093E800809133
:10243000E80082FF18C09091F3008091F2000297AB
:1024400031F48091F100813011F0863021F48091D7
:10245000F100809307028091E8008B778093E80079
:102460000E944B0A86CF809123048111E0CF81CF57
:102470008091F701813A09F07CCF8091FB01909126
:10248000FC01892B09F075CF8091E800877F80934C
:10249000E8008091E80080FFFCCF809104018093E8
:1024A000F1008091E8008E77D9CF8091F7018132D9
:1024B00009F05FCF8091E800877F8093E8000E9459
:1024C0004B0A8091FA018093F30153CF8091F70179
:1024D000813A09F04ECF8091E800877F8093E80031
:1024E0008091E80080FFFCCF8091F301D8CF803845
:1024F00089F0823849F58091FB018F70873020F593
:102500008093E9008091EB0085FB882780F9109289
:10251000E90007C09091CB03919592708091F401EE
:10252000892B9091E800977F9093E8008093F100C9
:102530001092F1008091E8008E7723C0811116C0BF
:102540008091F901813011F18091E80083FF0AC088
:102550008091E800877F8093E8008091EB008062A3
:102560008093EB00AA96E3E00C94D82C823061F7BC
:102570008091F901811589F01092E9008091E800BD
:10258000877F8093E8000E944B0ADECF81E0933082
:1025900009F080E08093CB03EFCF8091FB018F7037
:1025A0002FEF280F263080F68093E9002091EB0072
:1025B00020FFE2CF933031F48091EB008062809372
:1025C000EB00DACF9091EB0090619093EB0021E06B
:1025D00030E0A90102C0440F551F8A95E2F74093ED
:1025E000EA001092EA008091EB008860E8CF811148
:1025F000ABCF1091F9011F778091E3008078812B98
:102600008093E3008091E800877F8093E8000E9438
:102610004B0A8091E80080FFFCCF8091E300806846
:102620008093E30083E0111101C082E080932304D2
:102630008BCF8058823008F087CF4091F9015091BC
:10264000FA014C3D83E0580799F583E08A838AE2DA
:1026500089834FB7F894DE01139620E03EE051E203
:10266000E32FF0E050935700849120FF03C0829540
:102670008F703F5F8F708A30C8F0895C90E08D93D7
:102680009D932F5F243161F74FBF8091E800877FD2
:102690008093E8006AE270E0CE0101960E94F209A0
:1026A0008091E8008B778093E8004ECF805DE6CF85
:1026B0002091FB013091FC01852F992783309105F2
:1026C00009F160F48130910509F472C0029709F0B4
:1026D0003BCF8BE390E0E7E6F1E029C08132910542
:1026E00009F45AC0829709F02FCF2115310509F45A
:1026F00069C02130310509F027CF8BE790E0ECEA83
:10270000F0E015C0CA0199274130B1F1823091053E
:1027100009F43AC0892B09F017CFE4EFF1E0E49116
:102720008E2F90E0E4EFF1E0009709F40DCF2091B7
:10273000E800277F2093E8002091FD013091FE0101
:102740008217930708F49C0140E02115310509F038
:102750003EC041113CC08091E80082FDA1CF809134
:102760002304811509F49CCF853009F499CF809119
:10277000E80083FFF0CF94CFEAEDF1E0E4918E2FF3
:1027800090E0EAEDF1E0D0CFE4EBF1E0E4918E2FC0
:1027900090E0E4EBF1E0C8CF2115310571F0213074
:1027A000310509F0D1CE89E090E0E2E9F1E0BFCF58
:1027B00082E190E0E2EAF1E0BACF89E090E0E9E777
:1027C000F1E0B5CF80E490E0E7E2F1E0B0CF8091B6
:1027D0002304811509F464CF853009F461CF809119
:1027E000E80083FD5DCF8091E80082FDB4CF809149
:1027F000E80080FFAACF9091F3008091F2002115AC
:10280000310519F08830910550F041E0089709F042
:1028100040E08091E8008E778093E80096CF449165
:102820004093F1003196215031090196E8CF80386C
:1028300009F08ACE8091E800877F8093E80080913C
:10284000F5018093F10076CE81117ECE1091F901D1
:10285000123008F079CE8091E800877F8093E800FD
:102860001093F5010E944B0A111581F084E08093CA
:10287000230442E061EC81E00E94B90A42E261EC8B
:1028800082E00E94B90A809123045ECE8091E30029
:1028900087FDECCF81E0EBCFA0E0B0E0E2E5F4E132
:1028A0000C94B72C8901D42FC52F6B017C010E9499
:1028B0000C08A8016D2F7C2F88E090E00E94422E2A
:1028C00098014D2F5C2FB601C70100E20E94562DE2
:1028D000622F84E290E00E94302ECDB7DEB7E8E0B0
:1028E0000C94D32CE5E6F4E083E0808311828FEF33
:1028F000828380E883831482A2E6B4E012968C91EE
:102900001297836012968C93758123E030E04FEF2D
:1029100050E860E0868197810E944C140895809170
:102920006904833018F48F5F8093690420916504F3
:102930003091660440916704509168046091690485
:1029400070916A0480916B0490916C040E944C1405
:10295000089580916904811519F08150809369046C
:102960002091650430916604409167045091680499
:102970006091690470916A0480916B0490916C0479
:102980000E944C140895A3E0B0E0E9ECF4E10C944B
:10299000B52CE82ED62EF42EB22E9091650490FF21
:1029A00045C030916604381308C0809167048613CF
:1029B00004C080916804841729F0809164048260C7
:1029C00080936404E92FE695AE2FB0E0A859BE4F7E
:1029D0008C91809362049E7F923061F54F2D81E847
:1029E000F81608F040E89E012F5F3F4F6D2D8E2DA9
:1029F0000E947B074B8169818A810E94E90D3E2DEF
:102A000030936604D0926704F0926804B11471F0B8
:102A1000209165046091690470916A044D2D5F2DC9
:102A200080916B0490916C040E944C142396EAE010
:102A30000C94D12C823019F4F0906804E0CF8630E9
:102A4000F9F28930E9F28931D1F6E9519E2F91707E
:102A5000A92EE695F0E0E855FC4FE491C12C0E2F2D
:102A600010E060911701C61618F00E94BF0BC7CF87
:102A70002C2D30E0C09EC001C19E900D112470E04D
:102A80000E94FE2C8E2DA11017C0860F909115016B
:102A9000A901490F511D9A01220F331F240F351F21
:102AA000245E3C4F4F2D91E8F91608F040E86D2D5B
:102AB0000E947B07C394D5CF861BE8CFE5E6F4E000
:102AC000818121E043816281885F0E94C31408955F
:102AD000E5E6F4E0818121E04381628188500E9433
:102AE000C3140895E5E6F4E0628121E1620F08F481
:102AF0006FEF21E0438181810E94C3140895E5E6D0
:102B0000F4E0628121E1621B08F460E021E043818E
:102B100081810E94C3140895E5E6F4E0438121E138
:102B2000420F08F44FEF21E0628181810E94C314BB
:102B30000895E5E6F4E0438121E1421B08F440E01A
:102B400021E0628181810E94C3140895A8E0B0E071
:102B5000ECEAF5E10C94BD2C66EE7EEF80E090E0AF
:102B60000E944E2E60E082E090E00E94302E60E0F5
:102B700083E090E00E94302E109271041092700455
:102B800060E074E184E090E00E944E2E60E086E018
:102B900090E00E94302E6FEF87E090E00E94302E90
:102BA00040E050E0BA0188E090E00E94422E60E0F0
:102BB00084E290E00E94302E60E087E190E00E9485
:102BC000302E60E08CE090E00E94302E60E08DE0DE
:102BD00090E00E94302E19821A821B821C821D8274
:102BE0001E821F82188648E050E068E170E0CE0146
:102BF00001960E94202E40E050E0BA0180E290E071
:102C00000E94422E40E050E0BA018FE090E00E9426
:102C1000422E40E050E0BA0183E190E00E94422E53
:102C20002896E2E00C94D92CA1E0B0E0EAE1F6E1CC
:102C30000C94AF2C462E4A01522EC32E3701A82EDB
:102C4000880FBB08C5010E94392CD82E811509F4C4
:102C500075C0C50133E0880F991F3A95E1F7FC0173
:102C6000E35DFE4F2381422F50E0211511F041E03A
:102C700050E0835D9E4FFC0164817581635F7B4FF3
:102C8000CE0101960E94032EF401408151816281A0
:102C900073812FB7F8948091090490910A04A09150
:102CA0000B04B0910C042FBF841B950BA60BB70B24
:102CB00084369105A105B10538F4B301C8010E941D
:102CC0002F0899818917D1F1E42C042C000CFF08FE
:102CD000C7010E94392CD82E811106C0D12C8D2D10
:102CE0002196E0E10C94CB2CC70123E0880F991FBB
:102CF0002A95E1F7FC01E35DFE4F2381422F50E06E
:102D00006216710408F4A301835D9E4FFC01648187
:102D10007581635F7B4F852D9C2D0E94032EB3012F
:102D2000C8010E942F0899818913D8CF0E94D40925
:102D3000F4016083718382839383D1CFA301B801AF
:102D4000852D9C2D0E94032ECACFA4E0B0E0EBEAB3
:102D5000F6E10C94B72C6B0184E0E82EF12C0EE028
:102D600014E09E012F5F3F4F45E054E061E080E0BA
:102D70000E941416811561F049815A816B817C8112
:102D8000409301045093020460930304709304047D
:102D90004091010450910204609103047091040475
:102DA000F60140835183628373832496E8E00C9498
:102DB000D32CA1E0B0E0EFEDF6E10C94B62CEE24BC
:102DC000E394F12C03E114E09E012F5F3F4F4DEFA0
:102DD00053E063E082E00E941416082F811539F158
:102DE000D12C80E01DC0C090FC03CD0C2C2D30E018
:102DF000A90146505C4F7A01E1E0F0E0EC0FFD1FC5
:102E0000ED0DF11D1081FA019081191BB12E1B14DB
:102E10009CF0912F17FD90E0191B111118C0D3944D
:102E20009091F903D916F8F281110E94A00B802F1E
:102E30002196E9E00C94D22CBA94F70180818F5F3F
:102E4000808360E08C2D0E94F010802FE0CF1F5F08
:102E5000F70180818150808361E08C2D0E94F01009
:102E6000802FDBCFA4E0B0E0E8E3F7E10C94BC2CCA
:102E70004091F5035091F6036091F7037091F803C8
:102E80002FB7F8948091090490910A04A0910B0443
:102E9000B0910C042FBF841B950BA60BB70B11E050
:102EA00084369105A105B10578F10E94860BDC01FD
:102EB000CB010296A11DB11D89839A83AB83BC838C
:102EC00080914E0190914F01835F9B4F20914D0166
:102ED000422F50E0253010F044E050E0BE016F5F1B
:102EE0007F4F0E94032E84E090E00E94392C182F1F
:102EF000811551F00E94D4096093F5037093F60395
:102F00008093F7039093F803812F2496E3E00C94C9
:102F1000D82CCF92DF92EF92FF92CF93DF93CDB771
:102F2000DEB72B970FB6F894DEBF0FBECDBF88E09B
:102F3000E5E6F4E09E012F5F3F4FD90101900D922D
:102F40008A95E1F740916204909163048091640452
:102F500049879A878B87C090F103D090F203E09065
:102F6000F303F090F4039FB7F89440910904509153
:102F70000A0460910B0470910C049FBF4C195D0909
:102F80006E097F09E22F443651056105710510F481
:102F9000811511F18091560190915701835F9B4FEC
:102FA00020915501422F50E02C3010F04BE050E0C2
:102FB0006E2F732F0E94032E85E090E00E94392C23
:102FC000811569F00E94D4096093F1037093F203B4
:102FD0008093F3039093F4031092640481E02B96A2
:102FE0000FB6F894DEBF0FBECDBFDF91CF91FF903B
:102FF000EF90DF90CF900895A0E0B0E0E2E0F8E13C
:103000000C94AF2CFC016280448081E08483E8EA68
:10301000F2E07490E7E2F3E0E491C0916804C695B1
:10302000C158D0E0CC0FDD1FED2EFF24812C75E0C0
:10303000972EAA24AA94B12C55245A94E719CE2E7F
:10304000D12C80911701881638F00E94BF0BCDB7A4
:10305000DEB7E0E10C94CB2C082D10E083E068167D
:1030600068F4909EF001919EF00D1124E45FFD4FF5
:1030700080916604808380916704818341102DC014
:10308000909EF001919EF00D1124E45FFD4F13829C
:10309000128280911501800F912F911D9C01220FAA
:1030A000331F280F391F245E3C4F909EF001919EE4
:1030B000F00D1124E45FFD4F4281413808F040E8F3
:1030C000909EF001919EF00D1124E45FFD4F61810F
:1030D00080810E947B078394B4CF909EE001919EF3
:1030E000D00D1124C45FDD4F8B818115E9F0815033
:1030F0008B83589EC00111246C8170E00E94FE2CCD
:10310000FB01FF27E855FD4F8491E82FE7195E9EEC
:10311000C0011124B6010E94FE2C80916804689FB2
:10312000B00111247A83B5CF0E94D92DB5010E9438
:10313000122D8E159F050CF0ACCF83E0681688F039
:103140000E94D92DB5010E94122D88830E94D92D8D
:10315000209167042695622F70E00E94122D280F9F
:103160002983909EF001919EF00D1124E45FFD4FA4
:10317000128280916804893C58F088EC909EF0019E
:10318000919EF00D1124E45FFD4F8483838381CFF2
:103190008431A0F784E1F2CF60916504669570E018
:1031A0004BE050E088E091E00E94E92D892B19F472
:1031B00081E0809363040E94A30B9093E1038093CA
:1031C000E003809164048460809364040895909186
:1031D000650490FF3EC08115E9F18932E8F58F77EB
:1031E000282F220F809165048170282B209365047D
:1031F00080916404816080936404611581F0309152
:10320000660440916704509168046091690470916C
:103210006A0480916B0490916C040E944C1460913C
:103220006504669570E04BE050E088E091E00E9414
:10323000E92D892B99F00E94210881E08093E30316
:1032400020E04091680460916704809166040E94C8
:10325000C314089581E0C4CF88E2C2CF0E94CC1885
:10326000ECCF8091650486958F5F893208F081E00C
:1032700061E00E94E71808958091650486958A951B
:1032800009F488E261E00E94E718089590916504CE
:1032900090FF08C09695981728F0961718F40E948A
:1032A0003119089561E00E94E7180895A0E0B0E0A8
:1032B000ECE5F9E10C94AE2C8C01FC0184818115C4
:1032C00009F4C9C161E0C8010E94C306EC01F8011C
:1032D00085818115B1F080916E048272FE01E05308
:1032E000FC47E830F10568F4EA51F14D0C94262DC5
:1032F000811521F08FEF03C08115E1F381E00E9479
:103300001F0FF8015580511409F4CDC0D7FFCBC071
:103310000E94AE0B8093570490915804913029F489
:1033200081FF03C089E30E94721080916E04809334
:10333000560410926E0410927404809158048230E6
:1033400009F46EC0B8F4811164C082EE0E94B20F1D
:1033500017C0109258040E94180FD3CF81E08093B9
:103360005804F9CF82E0FBCF83E0F9CF84E0F7CFB8
:1033700085E0F5CF843009F467C0853009F469C071
:103380004E01E89497F8A12CB12CEFE3FCE93197BA
:10339000F1F700C00000409058045CE1C52ED12C2C
:1033A00067E0E62EF12C7AE0672E712CD501C4017E
:1033B0000C2C04C0B695A795979587950A94D2F7DB
:1033C000F82FFF703F2E511479F024E04212BCC553
:1033D0003AE0F31708F4B8C580915804823009F038
:1033E00049C082E60E94721080915804823009F030
:1033F00045C09AE08AEF830D391638F489E0830DD1
:1034000090E0B3010E94122D875A0E947210512C35
:10341000A2C560E070E088E193E00E943910B0CF6F
:103420008091570480FD03C083E50E94721082EEF4
:103430000E94B20F8FE39CE90197F1F700C00000F2
:1034400087E50E9472109CCF86EE0E94721088E180
:10345000F8CF60E070E08BE191E00E94391060E00D
:1034600070E085E290E00E94391060E070E088E250
:1034700090E0D3CF80E30E940011B6CF86EF830D9A
:10348000863028F080E3830D0E940011C0CF87E5CD
:10349000FACF843009F456C0853009F455C08091C4
:1034A000560480936E04F8018581811509F4DEC00D
:1034B000C137FCE7DF0709F4B5C0C2372CE7D207F4
:1034C00009F4CEC0C0373CE7D30709F05CC5809053
:1034D0005F019090600180915D0190915E0188167E
:1034E0009906C9F580915F048032A9F589E594E0D9
:1034F000EC01019628812032D9F38881811509F4E5
:103500009AC0813009F08BC099818A81913009F08D
:1035100052C022960E9472102196EFCF8CE20E9438
:1035200072108091570481FFBACF89E30E94721014
:10353000B6CF82EE0E9406108091570480FDAFCF77
:1035400083E5F4CF88E2F2CF60E070E088E290E0BB
:103550000E943910A4CF90925E0180925D0180E2BA
:1035600080935F04A12CB12C10925E043EE5E32E03
:1035700034E0F32EC0E0D0E04AE0442E512C612C20
:10358000712CC501B401A30192010E94962E605DC9
:10359000603339F4209729F089288A288B2809F488
:1035A00060E2F70162937F0149015A012196C5301B
:1035B000D10539F79BCF923021F422960E94B20FA9
:1035C000ABCF933021F422960E940610A5CF943001
:1035D00011F02196A1CF229620E030E06AE0AE0102
:1035E0004F5F5F4F8053990B8A30910568F021152A
:1035F000310509F491CF8FE99FE00197F1F700C001
:10360000000021503109F3CF629FF001639FF00D5C
:1036100011249C012E0F3F1F8981EA01E0CF0E94F7
:1036200000117ACF80915F0190916001059690938F
:10363000600180935F01809175048770811559F056
:10364000F8018581811539F08091BC0482FF03C0A7
:1036500082E00E944404CDB7DEB7E1E10C94CA2CAD
:1036600080915F01909160010597E1CFFE01E851E3
:10367000FC47E730F10508F0DDC0E251F14D0C9454
:10368000262D26E241EE61EE0E949210D4CF27E271
:1036900045EE65EEF9CF26E241EE60EEF5CF27E28A
:1036A00045EE64EEF1CF26E241EE62EEEDCF27E289
:1036B00045EE66EEE9CF28E241E0EBCF8091BB0416
:1036C00081608093BB046091BB047091BC0484E072
:1036D00090E00E944E2E0E945D11ADCF8091BC04FF
:1036E00088608093BC04EFCF8091BB048260E9CFF7
:1036F0008091BB048460E5CF8091BB048860E1CFFA
:103700008091BC048160EDCF8091BC048260E9CFE0
:103710008091BB048061D5CF8091BB048062D1CF02
:103720008091BB048064CDCF0E945D118091BB0469
:103730008068C7CF8091BB048C60C3CF8091BC04EC
:103740008360CFCF8091BB048E7FBBCF8091BC04C0
:10375000877FC7CF8091BB048D7FB3CF8091BB049F
:103760008B7FAFCF8091BB04877FABCF8091BC04B0
:103770008E7FB7CF8091BC048D7FB3CF8091BB0487
:103780008F7E9FCF8091BB048F7D9BCF8091BB04A8
:103790008F7B97CF0E945D118091BB048F7791CF73
:1037A0008091BB04837F8DCF8091BC048C7F99CFA7
:1037B0008091BB0482FB992790F921E0922790FB2E
:1037C00082F990FB83F97DCF8091BC04982F90956E
:1037D00090FB80F990FB81F984CF9091BB04892FF5
:1037E0008F7B96FF80646DCF0E945D119091BB042A
:1037F000892F97FB87F9805864CF61E08EE090E0D5
:103800000E94302E60CF60E0F9CF9091BB04892FE9
:103810008F7E94FF806155CF9091BB04892F8E7F5E
:1038200090FF81604ECF9091BC04892F877F93FFDA
:10383000886057CFC6319CE7D90709F590916E048F
:10384000811599F0892F8A7A91E0811101C090E069
:103850009093610465E3811101C069E28EED91E00E
:103860000E9493080E943E0FE6CE8091610481156C
:1038700021F085E30E943704F5CF89E2FBCF811167
:1038800089C080916E048272FE01E052F847E531F2
:10389000F10508F094C0EB50F14D0C94262D809169
:1038A000650480FF1EC0282F2E7F20936504309171
:1038B00066044091670450916804609169047091B6
:1038C0006A0480916B0490916C040E944C140E94D5
:1038D0002108809164048160809364040E94BF0B7E
:1038E000AACE81608093650461E086950E94E71806
:1038F000A2CE4CE359E161E379E10E9428089BCE16
:1039000041E359E16CE379E1F8CF48E655E16EE532
:1039100075E1F3CF4EE555E168E675E1EECF4FE78F
:1039200055E162E775E1E9CF42E755E16FE775E1FF
:10393000E4CF49E955E16CE875E1DFCF4CE855E1AA
:1039400069E975E1DACF49EA54E16FE874E1D5CF6E
:103950004FE854E169EA74E1D0CF61E081E0C6CF7D
:1039600065E082E00E94461966CE68E086E0FACF04
:103970006EE089E0F7CF64E18FE0F4CF67E185E1A5
:10398000F1CF61E088E1B2CF62E289E1EBCF68E29A
:1039900083E2E8CFCA35ECE7DE0709F485C008F01A
:1039A0005CC0C1302CE7D20709F47CC0C3303CE7CF
:1039B000D30709F471C0C115DC4709F460C0F801F0
:1039C0008581E080F180811509F472C0C7010E94F1
:1039D0008F06C82F682FC7010E94C403B7018C2F20
:1039E0000E9473040E947805D82FC92FF801B58072
:1039F000A680A2942FE0A222809175048770811581
:103A0000F1F0EB2CB114E1F0892F807F803451F07C
:103A100080E28D0F883098F0A11004C0892F807E3D
:103A2000803269F08091BC0482FF09C082E00E946C
:103A30004404809175048770EE24E3948111E12C95
:103A40008C2F82958F70C82ED12C8C3008F095C0A9
:103A5000F601E65FF04D0C94262DCB359CE7D90797
:103A600029F1CC35DC4709F0AACF8091BC0482FB58
:103A7000882780F991E089270E94010FA0CF0E943A
:103A80005D11FFEF24E33CE0F15020403040E1F7CE
:103A900000C000000E94440E6FEF7FEF80E090E0D6
:103AA0000E944E2E0E94841181E0E6CF80E0E4CF98
:103AB000C7010E94FA03C82F91CFFC2FFF70FF2E81
:103AC000C03118F0F29490EFF922B114B9F0F1146A
:103AD00069F080E28D0F883010F0D11109C080911B
:103AE0006E048F2980936E040E943E0F8D2F43C079
:103AF000809174048F2980937404F6CF8D2F0E94D7
:103B00000610F114D1F180E28D0F883010F0D11140
:103B100004C08F2D0E94600406C0F094809174044C
:103B20008F21809374040E943E0F27C02C2F2F708A
:103B3000F22EC07FC03219F0F29480EFF822D11536
:103B400051F0D13009F491C0B11409F49BC0A11413
:103B500009F442C0CBCF8091BC0482FD39C0B114BE
:103B600089F1F11439F080916E048F2980936E04ED
:103B70000E943E0F80E00E94B20F28E0C21AD108D6
:103B800034E0C316D10410F40E94AE0BE114A9F086
:103B90008091750480FD11C0F80115828695869587
:103BA00086950E94A203C8010E945619809175044F
:103BB0008695869586950E94B20360E0C8010E94B2
:103BC000C30649CD80E00E940610F114B1F2A1CFE6
:103BD000B11469F1A11004C08F2D0E949E0FCDCFAA
:103BE00031E0A31210C0C0916D048F2D8C23F81604
:103BF00021F20E94AD089093790480937804CF2934
:103C0000C0936D04BACF83E0A812B7CF8F2D0E9466
:103C10009E0F8F2D0E94D10880916F049F2D9823B5
:103C2000F91609F4AACF8F2980936F04A6CFA110AB
:103C300012C08F2D0E948C0F8F2D0E94D108809171
:103C40006F049F2D9823911509F497CFF094F822D3
:103C5000F0926F0492CF91E0A9128FCF80916E0401
:103C60008F21811509F489CFE4CFB11429F0E2E066
:103C7000AE1608F082CFB0CFA1107FCF8F2D0E945B
:103C80008C0F7BCFA114D1F3D93349F4FFEF27EE8A
:103C900033E0F15020403040E1F700C000008D2FAC
:103CA0000E9406106ACF8C2F8695869583708115A9
:103CB00069F0813009F061CF8D2F9C2F9370B11086
:103CC00002C080E090E00E946D0857CF8D2F9C2F9E
:103CD0009370B11002C080E090E00E9447084DCF81
:103CE0006B2D8D2F0E940F0948CF8C2F837081116F
:103CF00040C0B11042CF4D2F429546954770440FBA
:103D0000440F2D2F2F7030E0042E02C0220F331FDE
:103D10000A94E2F780E090E0D4FF09C08FE090E0E1
:103D200002C0880F991F4A95E2F780959095C69535
:103D3000C695C370C230A1F0C33079F040917004D1
:103D400050917104C13039F0822B932B8423952339
:103D50000E94980312CF242B352B822B932BF8CF64
:103D6000822B932B2091700430917104822793272A
:103D7000EFCFB11491F1C0FF00CF4D2F4295469582
:103D80004770440F440F2D2F2F7030E0042E02C0D7
:103D9000220F331F0A94E2F780E090E0D4FF09C0BD
:103DA0008FE090E002C0880F991F4A95E2F7809556
:103DB0009095C695C695C370C230C1F0C33099F0D6
:103DC0004091720450917304C13059F0822B932BAF
:103DD000842395230E949D03D0CE823008F4CDCE5B
:103DE000CCCF242B352B822B932BF4CF822B932BF0
:103DF000209172043091730482279327EBCFCF7008
:103E0000B11429F08C2F0E94A2038D2FE6CE8D2FA6
:103E10000E948C0F8C2F0E94B203AFCED23F09F4C8
:103E20003EC060F4D03FB9F0D13F81F0B11409F445
:103E30007BC0A1105BCE8C2F8F7135C0D33FB1F109
:103E4000D43FA1F78091BC0482FD3EC08C2F8F71BE
:103E5000B11409F328C0B11499F0A1108ECECF711E
:103E600081E090E0FC0102C0EE0FFF1FCA95E2F76F
:103E7000EF0180917204909173048C279D27AACF43
:103E8000F2E0AF1608F079CECF7181E090E09C01AE
:103E900002C0220F331FCA95E2F7E901EACF8C2F47
:103EA0008F71B110B8CF0E94A20367CE80E090E07E
:103EB000B11409F48FCFCF7181E090E002C0880F78
:103EC000991FCA95E2F786CFB114E9F08091750485
:103ED0008770843061F41092750410927704109208
:103EE00076048C2F8F710E94B203E12C46CE33E012
:103EF000A316D8F7CF718C2F0E94A20363E08C2FFA
:103F00000E94B908F2CF83E0A81650F01092750411
:103F1000109277041092760464E08C2F8F71F0CFAA
:103F200081E00E944404E1CFA11459F0D93309F093
:103F3000B6CE9FEFE7EEF3E09150E040F040E1F7BE
:103F4000ACCE8C2F8F7167CF31104ECA84E0E8164B
:103F5000F1040CF449CAE1E0EE1AF108F4E0CF1ADA
:103F6000D1082FEFE216F20609F020CA809158041A
:103F7000823009F4DECA08F08CCA8111CFCA82EE01
:103F80000E9406108CCAFE01E851FC47E730F1059B
:103F900008F473CB109260049E0130572332310530
:103FA00008F048CC84E090E00E941A2E9093BC0464
:103FB0008093BB04FE01E150F047E232F10508F0C6
:103FC0007DCBEA5EF04D0C94262D8091BA048031B1
:103FD00078F48091B904811559F0E0917B04209127
:103FE0007A043091B5044091B40457E02E1301C017
:103FF00008956E2F70E05E9FF0011124DF01A45838
:10400000BB4F14968C911497811581F111968C9168
:10401000119783132BC08C91841328C015968C9113
:104020001597811123C012968D919C91A091B60491
:10403000B091B7048A1B9B0BA0915F01B091600106
:104040008A179B0798F48091BA048F7080618093DF
:10405000BA04EE57FB4F80818F708061808384EBC0
:1040600094E00E9456190E942D040895FB01319698
:10407000E770BCCFADE0B0E0E0E4F0E20C94B22C2D
:104080008C0186E0F801DE01189601900D928A9568
:10409000E1F7F801E080F580A280B380C48084EB72
:1040A000882E84E0982E7090B804711020C0C1143E
:1040B000D9F0F11409F421C1C8010E94F20681155A
:1040C00009F41BC187E0F801D40101900D928A9593
:1040D000E1F7F1E0CF1206C08091B4049091B504ED
:1040E0000E94E3060E94E51FFF24F39456C0D0907F
:1040F000B9048091B6049091B7049501281B390B3F
:10410000C90120915F0130916001D11409F4BAC056
:104110008217930708F090C0C11431F39091B50451
:10412000C1808091BA04803108F058C0C91214C00F
:104130009091B4049E1110C0F1104AC08F7080613C
:104140008093BA0484EB94E00E9456198091BA04DB
:10415000F8018683F12C21C0F1103AC040E06C2DAB
:104160008E2D0E94440B40E06C2D8E2D0E94440B3E
:10417000F82E8111EFCF888599850E94E306292FBB
:1041800022952F70903470F49F702230A0F091151A
:10419000B1F0F8019681903190F48F2D2D96EDE0DD
:1041A0000C94CE2C2A5F2F70223068F0C8010E9438
:1041B0005619FD2CF2CF911511F0811571F3805E27
:1041C000883058F3F3CF803F40F3815F8330F9CFDD
:1041D0008091BA0481608093BA04BCCFC91207C031
:1041E0009091B4049E1103C0F11409F46FC0C8018A
:1041F0000E94F206811509F480C0F11409F47DC013
:104200008091BA04803278F02091B4043091B504E2
:104210003A832983BC82AB827D821E828F83CE014A
:1042200001960E94561987E0F801A4EBB4E00190D2
:104230000D928A95E1F756CF8091BA04803150F4FF
:1042400084EB94E00E94561987E0F40111928A955C
:10425000E9F780CFC11409F447CF2091B5049181CB
:104260002913C5CF9091B4049E11C1CFF110BFCFD7
:104270008683C8010E94561987E0F40111928A953D
:10428000E9F732CF82179307F8F6C11409F42CCF5F
:10429000F11499F13091B5042181321324C0209199
:1042A000B4042E1120C08E3B9105A0F48091BA0475
:1042B00080FD10C0803170F08683982F907F903FF2
:1042C00031F0982F907F905F8F70892B8683C80183
:1042D0000E94561987E0F801A4EBB4E001900D921A
:1042E0008A95E1F701CFC8010E94F20681119BCFA8
:1042F0008091BA0481608093BA04C8010E94561963
:10430000F3CEABE1B0E0E7E8F1E20C94BC2C4E8BCD
:104310005F8B688F798F8A8F9B8F911110927404B5
:104320001D8A86E0FE017696DE011F9601900D92B1
:104330008A95E1F78091BC0482FF1FC00E94AD08FE
:104340002091760430917704821B930B8838934137
:1043500038F08091750482FD03C082E00E9444041D
:104360000E94AD082091780430917904821B930B50
:104370008838934110F00E9468048B89811529F0D8
:1043800061E0CE010F960E94C30687E0FE013F96D2
:10439000DE01189601900D928A95E1F7CE010896FC
:1043A0000E943A20811110C087E0FE013896DE019C
:1043B000119601900D928A95E1F720917A0440912F
:1043C0007B048C8581110BC017E080917B04909158
:1043D0007A0489132DC06B96E3E00C94D82C30E05E
:1043E000C9010196877099274817190671F40E9430
:1043F0005D1110927A0410927B0487E0E4EBF4E004
:10440000DF011D928A95E9F7DFCF97E0929FD001F7
:10441000939FB00D1124A458BB4FFE01319601901B
:104420000D929A95E1F780937A040E942D04CCCFE7
:10443000189FC001112484589B4F0E943A20811577
:1044400051F280917B0490E00196877099278093C8
:104450007B04BBCFA6E0B0E0E0E3F2E20C94BB2C1F
:104460000E94AD088C018091290490912A04801744
:10447000910779F019821A820E94AD08BC01498126
:104480005A8180E090E00E94812110932A040093D9
:1044900029042696E4E00C94D72CA3E1B0E0E3E5F0
:1044A000F2E20C94B22CFE013C9688E0DF011D92F2
:1044B0008A95E9F78EE1A82E81E0B82E8F014F0191
:1044C000EE24E394F12C2EE1C22E21E0D22EF50150
:1044D00081915F018F3F09F441C0F894E82FE29584
:1044E000EF70F0E021A18F70A70102C0440F551FAB
:1044F0008A95E2F7CA01922F982B91A392A18095F9
:10450000892382A3789400C0E8E1F1E031E0712CC6
:1045100021912F3F89F0A22FA295AF70A05EB0E04D
:104520008C9190E02F7002C0959587952A95E2F7BF
:104530008170811509F49AC080E0782A330FCE1675
:10454000DF0631F7F501319780818F3F11F00E942E
:104550001C0750EA5A95F1F7D8017C920F5F1F4F64
:10456000B2E2AB16B1E0BB0609F0B1CF48E050E0D3
:10457000B4018EEB93E00E94F62D892B09F078C0F0
:104580000091C7038091EF018115F1F08091ED0159
:104590009091EE010E94E0090597B0F010E00453FD
:1045A0001C4F44E050E06EEB73E0C8010E94F62D12
:1045B000892B41F084E0EEEBF3E0D80101900D92FD
:1045C0008A95E1F71092EF010E94630BE091C70317
:1045D0009E012F5F3F4F7901811509F492C084E05D
:1045E000D9011D928A95E9F70E2F10E004531C4F54
:1045F0008091F0018A3008F04FC045EA56E1B701DA
:10460000C8010E94C70E811509F469C049ED56E141
:10461000B701C8010E94C70E811509F460C042E3CA
:1046200057E1B701C8010E94C70E811509F457C0B0
:1046300049E857E1B701C8010E94C70E811509F486
:104640004EC01092F0018091C60390E044E050E02B
:10465000B70184539C4F0E94F62D21E02093EC017A
:10466000892B79F56396EDE00C94CE2C832F65CFE2
:1046700088E0F401AEEBB3E001900D928A95E1F78A
:104680000091C70381E08093EF010E94AD089093F1
:10469000EE018093ED017ACF8091EA019091EB01D8
:1046A0000E94E009843F914008F0A7CF8091EC017F
:1046B0008115C1F284E0F70111928A95E9F7109211
:1046C000EC01E091C603F0E0E453FC4F89819A814C
:1046D000AB81BC8180839183A283B383C3CF80915C
:1046E000F0018F3F39F40E94AD089093EB01809365
:1046F000EA01DCCF8F5F8093F0018A3008F4A3CF0A
:10470000F2CFF0E0E453FC4F80819181A281B3812C
:1047100080930E0490930F04A0931004B09311049F
:1047200064E070E08EE094E00E942F0880930D0416
:104730004091E90350E06091E80370E066507C4FDF
:10474000C7010E94032E89818093130461E070E009
:10475000C7010E942F088093120480901404909047
:104760001504A0901604B09017048091E601909172
:10477000E701A091E801B091E90188169906AA061F
:10478000BB06D1F08092E6019092E701A092E80189
:10479000B092E9010E94630B81110EC00E94D409FE
:1047A000861A970AA80AB90A8092250490922604CC
:1047B000A0922704B09228048BE0E8E1F4E0D7014E
:1047C00001900D928A95E1F7809118048695F090FA
:1047D0001904E0901A04D0901B0400912104109158
:1047E000220410922204111509F43CCF10FF0BC0D3
:1047F00029819091650420FF1AC09160909365040F
:1048000060E00E94E71811FF06C020E04D2D6E2DDC
:104810008F2D0E94C31412FF04C00115A9F00E943D
:10482000CC1813FF1FCF81E08093E3031BCF9E7F43
:10483000909365040E9421088091640481608093B4
:1048400064040E94BF0BDFCF0E942108EACFCDB7DE
:10485000DEB728970FB6F894DEBF0FBECDBF85B781
:10486000806885BF85B7806885BF84B7877F84BF30
:104870000FB6F894A89580916000886180936000DD
:10488000109260000FBE80E890E00FB6F89480931D
:104890006100909361000FBE8AE197E09093DD0183
:1048A0008093DC010E949A0A0E94E90A8091E2004A
:1048B00084608093E200789480912304811599F0BC
:1048C0008091E9001091EC001795112717958F70D2
:1048D000182B1092E9008091E80083FD0E949A1144
:1048E0001F701093E90082E084BD93E095BD9AEFBC
:1048F00097BD80936E0010922504109226041092AA
:1049000027041092280484988C988FE891E00197EE
:10491000F1F700C000008FB1829581708093220171
:1049200080912201811107C18BE1809313018BE1FA
:10493000809314010E94630B81110E944A2B909175
:10494000220181E0292F28272093E8039093FC037C
:10495000909122018093E903909122018093F903C1
:1049600080912201811106C086EF80932C0187EF90
:1049700080932B0180912C01E82FE295EF70A1E24A
:10498000AE0FB0E04C918F7021E030E0B90102C071
:10499000660F771F8A95E2F7CB01962F90959423A7
:1049A0009C93EE5DF0E09081892B808380912B01B8
:1049B000E82FE295EF70A1E2AE0FB0E04C918F705E
:1049C000B90102C0660F771F8A95E2F7CB01962FD7
:1049D000909594239C93EE5DF0E09081892B8083E9
:1049E0008FE891E00197F1F700C000001091E90312
:1049F0006CE271E04BE251E02AEEE22E23E0F22E6F
:104A0000FB018E2F861B811708F497C0809122012D
:104A100081111EC081E380931E0183E380931F01F7
:104A200082E38093200186E38093210186E0E1E622
:104A3000F1E0DE01119601900D928A95E1F786E092
:104A4000FE013196A8E1B1E001900D928A95E1F75F
:104A50008091220191E08927880F880F8093C703F6
:104A600094E0981B9093C6030EE111E092E2E92EC8
:104A700091E0F92EF80181918F018F3F11F00E9492
:104A80001C07E016F106B1F708E111E08EE1E82E0F
:104A900081E0F82ED8018D918D018F3F11F00E9499
:104AA0001C07E016F106B1F788E0ECECF3E0DF015B
:104AB000282F1D922A95E9F7EEEBF3E0DF011D9216
:104AC0008A95E9F780E090E00E941A2E863E9E4F7C
:104AD00011F00E94A61582E090E00E940C2E8093B7
:104AE000D40384E090E00E941A2E9093BC0480933B
:104AF000BB040E944D22EFEFF6E721E0E150F040C9
:104B00002040E1F700C000000E944D22EFB1E29585
:104B1000E17081E0E827EE0FEE0FF0E0E453FC4F88
:104B2000808185FF32C06FEF7FEF80E090E00E94D0
:104B30004E2E0E94440E80E0F8CE0191802F829587
:104B40008F70805E90E0DC012C91DA013D91AD0127
:104B5000832F82958F70805E90E0DC018C9190E0D5
:104B60003F7002C0959587953A95E2F78170880F5E
:104B700030E00F7002C0359527950A95E2F7217055
:104B8000822BD7018D937D013CCF83E090E00E9482
:104B90000C2E90E00E9498038CE090E00E940C2E76
:104BA00080935804843009F415C1811509F416C1A5
:104BB000813009F415C11092C80384E08093580431
:104BC0008091C903811192C080E090E00E941A2E6A
:104BD000863E9E4F21F00E94A6150E94721488E026
:104BE00090E00E94142E6B017C0184E290E00E9410
:104BF0000C2E282F30E040E050E060E070E080E0D4
:104C000090E000E20E943B2DE22FA32EB42EB52FA0
:104C1000A62FF72F9701860140E050E0BA01EC295A
:104C2000A12AB22AB32BA42BF52B862B972BE0932A
:104C30006504A0926604B0926704B0936804A093E0
:104C40006904F0936A0480936B0490936C048091E0
:104C50006404836080936404E230C8F50E94721497
:104C600088E090E00E94142E6B017C0184E290E0C9
:104C70000E940C2E282F30E040E050E060E070E011
:104C800080E090E000E20E943B2D5901B42FA52F57
:104C9000F62FE72F9701860140E050E0BA01AC28DB
:104CA000B12AB22BA32BF42BE52B862B972BA092AA
:104CB0006504B0926604B0936704A0936804F0930F
:104CC0006904E0936A0480936B0490936C040E94DF
:104CD0000C080E9421088091650480FF04C060E0F8
:104CE00086950E94E71881E08093C9030E94630BB8
:104CF000811102C00E944D2B83E291E090932C041D
:104D000080932B04FDEDCF2EF3E0DF2EA4E06A2E7E
:104D1000712CCE010196B8E1AB2EB12C8F83988710
:104D200080912304853049F480912304853009F46F
:104D300059C00E945D110E94AE0B0E944D2205EDEC
:104D400013E0ECECEE2EE3E0FE2ED701F80191919A
:104D50008D91CE16DF0609F495C09817C1F30E9415
:104D6000630B282E912CD7018D907D01F801319095
:104D70008F01381441F13824512C44244394842D5C
:104D800083218115C1F02114B1F059829A820E94C9
:104D9000AD089C838B83F1E0FD8391E0842D882115
:104DA000811101C090E09E8349815A816B817C8191
:104DB0008D810E9481215394440C26E05212DFCF52
:104DC000F80131978082939448E09412CCCF0E94EE
:104DD000860B5CC080E08093C803F2CE81E0FBCFFD
:104DE00082E0F9CF80912304843011F11092CA033C
:104DF00060E40FB6F894A895A09260000FBE60938F
:104E0000600083B7817F846083BF83B7816083BF85
:104E10007894889583B78E7F83BF0FB6F894A89552
:104E200080916000886180936000109260000FBEE6
:104E30008091CB03811509F477CF0E944D22ECECD1
:104E4000F3E084ED93E02191211104C08E179F07B8
:104E5000D1F76ACF80E189BD82E189BD09B400FE46
:104E6000FDCF8091D8008F7D8093D8008091E000A5
:104E700082608093E0008091E00081FDFCCF0E9481
:104E80005D1152CF98136BCF0E942A220E94630BB0
:104E900080916304811509F46CC080916204E091F3
:104EA0006504E695E81BE093E2038F3009F49AC0AD
:104EB00008F062C0863009F47EC0893009F486C0EB
:104EC000823009F46DC000ED17E075E3E72E77E05E
:104ED000F72E8091E303811561F01092E3030E94A5
:104EE000A30B9093E1038093E0031092E5031092EB
:104EF000E4030E94A30B9C018091E0039091E103E5
:104F0000A901481B590B4F3F5F4798F54091DF03BC
:104F10004115B1F01092DF034091DD035091DE03A3
:104F2000241B350B2F3F3F4758F4405D5A485093A0
:104F3000DE034093DD032091640428602093640421
:104F40008090E4039090E503800F911F9093E1031C
:104F50008093E00380EE93E0F70109958091E403EC
:104F60009091E503892B29F4892819F081E0809339
:104F7000DF03E12C912CCFC0883109F44FC083327C
:104F800009F43CC0853109F09ECFF0E0E055FB4FBD
:104F9000E4910E2F10E025EDE22E2CE0F22E99CFB9
:104FA000F0E0E454FB4FE4910E2F10E060E2E62EB7
:104FB0006EE0F62E8ECFF0E0E754FB4FE4910E2F1B
:104FC00010E054E3E52E5EE0F52E83CFE695F0E0A9
:104FD000EA54FB4FE4910E2F10E041E1E42E4CE047
:104FE000F42E77CFE695F0E0ED54FB4FE4910E2FD1
:104FF00010E03FE4E32E3CE0F32E6BCF8E2F63E016
:105000000E94E42CE92FF0E0E355FB4FE4910E2FD2
:1050100010E09CEFE92E97E1F92E5BCF08E210E05B
:1050200088E5E82E8DE0F82E54CF0E2D10E0F80123
:10503000E45DFE4F4081E42FE295EF70E05EF0E02A
:105040002081F801E55DFE4F3081E32FE295EF709E
:10505000E05EF0E0808190E03F7002C0959587951A
:105060003A95E2F78170880F30E04F7002C03595B5
:1050700027954A95E2F72170822BD801A651BC4FA3
:10508000EC919E2F9370891709F444C0EE0FEE0F38
:10509000E82BEC93F090E803FE0CEF70F0E0EC5698
:1050A000FE4F0A511C4F8081D8019C91890F8C932F
:1050B00020E0843084F0EF2DF0E0E650FC4F80815A
:1050C0008F5F80830E94630B811521F060E08F2D3C
:1050D0000E94F01021E0F80180818D3F84F4EF2DD3
:1050E000F0E0E650FC4F8081815080830E94630B8A
:1050F000811521F061E08F2D0E94F01021E0D80190
:105100008C91082E000C990BB3010E94122DF8010E
:105110008083922AE3948091E903E81608F485CF0E
:1051200091100E94A00B86E0E0E5F4E0AF81B88525
:1051300001900D928A95E1F7109252041092530457
:1051400010925404109255048B819C81892B8115F7
:1051500009F44BC08091EE039091EF030E94E009A7
:105160009C0180914E04811509F4C9C02531310597
:10517000E0F18F3F19F08F5F80934E041B81111572
:1051800059F00E94360791E011160CF09FEF899FAD
:10519000802D1124809352041C81111559F00E9416
:1051A000360791E011160CF09FEF899F802D112496
:1051B00080935304309152043115B9F02091530477
:1051C000211599F045EB3403C0011124892F911169
:1051D00001C081E08093520465EB26039001112405
:1051E000311509F47FC0309353048D819E81892B42
:1051F000811509F44AC08091EC039091ED030E945F
:10520000E0099C0180914D04811509F473C021359A
:105210003105D8F18F3F19F08F5F80934D041D81C8
:10522000111559F00E94560791E011160CF09FEFEE
:10523000899F802D1124809354041E81111559F0EB
:105240000E94560791E011160CF09FEF899F802D68
:10525000112480935504309154043115B1F02091FC
:105260005504211591F075EB3703C0011124892FE6
:10527000911101C081E08093540445EB2403900117
:105280001124311599F13093550446E050E06F81B7
:10529000788580E594E00E94F62D892B61F4809159
:1052A000520490915304892B90915404892B90912E
:1052B0005504892B81110E94E70886E0EF81F8856B
:1052C000A0E5B4E001900D928A95E1F70E94AE0B43
:1052D0009091F003891709F423CD8093F0030E9485
:1052E000D4091ECD81E0809353047FCF81E0809369
:1052F0005504CBCF2B30310508F08ECFC6CF2B30E5
:10530000310508F038CF71CF1F921FB61F921124BC
:105310008F939F93AF93BF938091CA03811113C062
:105320008091090490910A04A0910B04B0910C049F
:105330004196A11DB11D8093090490930A04A09386
:105340000B04B0930C04BF91AF919F918F911F906C
:105350001FBE1F90189578941F921FB61F9211249C
:105360008F939F93AF93BF938091090490910A0408
:10537000A0910B04B0910C040196A11DB11D809366
:10538000090490930A04A0930B04B0930C04BF91FA
:10539000AF919F918F911F901FBE1F9018951F92E4
:1053A0000F920FB60F9211242F933F934F935F9359
:1053B0006F937F938F939F93AF93BF93EF93FF93DD
:1053C0008091E10082FF09C08091E20082FF05C068
:1053D0008091E1008B7F8093E1008091DA0080FF73
:1053E00024C08091D80080FF20C08091DA008E7F99
:1053F0008093DA008091D90080FF9BC080E189BD55
:1054000082E189BD09B400FEFDCF81E080932304D1
:105410008091F601811109C00E949A0A0E94E90A4E
:105420008091E20084608093E2008091E10080FF3F
:1054300017C08091E20080FF13C08091E2008E7F50
:105440008093E2008091E20080618093E20080918D
:10545000D80080628093D80019BC85E08093230433
:105460008091E10084FF29C08091E20084FF25C083
:1054700080E189BD82E189BD09B400FEFDCF809144
:10548000D8008F7D8093D8008091E1008F7E80933B
:10549000E1008091E2008F7E8093E2008091E20043
:1054A00081608093E2008091F501811509F447C085
:1054B00084E080932304809123048091E10083FFA2
:1054C00027C08091E20083FF23C08091E100877FA5
:1054D0008093E10082E0809323041092F501809193
:1054E000E1008E7F8093E1008091E2008E7F8093C7
:1054F000E2008091E20080618093E20042E060E09F
:1055000080E00E94B90A8091F00088608093F000EA
:10551000FF91EF91BF91AF919F918F917F916F918B
:105520005F914F913F912F910F900FBE0F901F9061
:10553000189519BC109223041092F60176CF809131
:10554000E30087FF02C083E0B4CF81E0B2CF1F92B7
:105550000F920FB60F921124FF920F931F932F9368
:105560003F934F935F936F937F938F939F93AF93EB
:10557000BF93CF93DF93EF93FF9309EE10E0F80111
:105580008081C091EC00C795CC27C7958F70FC2E09
:10559000F82A1082C0EFD0E08881877F88837894D2
:1055A0000E949A11F8011082888188608883CF2D2B
:1055B000CF70C083FF91EF91DF91CF91BF91AF91F9
:1055C0009F918F917F916F915F914F913F912F911B
:1055D0001F910F91FF900F900FBE0F901F90189585
:1055E0008EE14A9B02C08A95E1F74A9BFECF08955F
:1055F0005A9880E28A95F1F75A9A0895FC013BE0A7
:105600003A95F1F798E020E080E031E040E14A95FA
:10561000F1F7880F4A9B02C08160232742E04A9538
:10562000F1F7000040E14A95F1F79A9579F790E19A
:105630009A95F1F799B132E03A95F1F7000040E11F
:105640004A95F1F792FB992790F992272081920FC2
:1056500090830895A1E0B0E0E0E3FBE20C94B92C64
:1056600019828C017C01E60EF11C0E151F0541F418
:1056700081E09981911180E02196E6E00C94D52C8F
:105680000E94F02ACE0101960E94FE2AF801819321
:105690008F01EBCF529A5A9A089552985A9AEA9AE1
:1056A000E9E6F0E080818F7C808308956150770B7C
:1056B00091E001C0990F6A95EAF7692F90E021E027
:1056C000611108C0911599F05A9A80E28A95F1F714
:1056D0005A980895362F3823311539F05A9A92275F
:1056E00030E23A95F1F76695EBCF5A98F9CF5A9890
:1056F000ECCFFF920F931F93CF93DF93EC018C01BC
:10570000060F111DC017D10729F4CDB7DEB7E5E0AC
:105710000C94D62CF9900E94F82A68E08F2D0E94F4
:10572000562BF0CF1F920F920FB60F9211240F93AA
:105730001F932F933F934F935F936F937F938F9319
:105740009F93AF93BF93EF93FF93CF93DF930F920A
:10575000CDB7DEB719820E94F02ACE0101960E94D1
:10576000FE2A082F069506950695982F9295957016
:10577000202F2570920F292F237096959695920FC2
:10578000982797708981892B811509F05CC00730B3
:1057900008F059C080E18A95F1F75A9A529A82E04E
:1057A0008A95F1F700C05A9888E0089F800111247B
:1057B000D801A35DBE4F1696ED91FC9117973097D7
:1057C000A9F06091A4017091A50114962D913C91CE
:1057D0001597260F371F11968D919C911297680F80
:1057E000791F13964C9113978C910995F801E35DFD
:1057F000FE4F6381611551F02091A4013091A50104
:1058000084819581820F931F0E94792B0E94F82A30
:1058100080E18A95F1F75A9852985A9A80E18A95D0
:10582000F1F7F801E35DFE4F6081611551F02091C1
:10583000A4013091A50181819281820F931F0E9462
:105840002A2B0E94F02A0F90DF91CF91FF91EF91C8
:10585000BF91AF919F918F917F916F915F914F9188
:105860003F912F911F910F910F900FBE0F901F909E
:1058700018950F931F93CF93DF938C0107970CF02C
:1058800064C0F894529A5A9885E08A95F1F700001E
:10589000C02FC695C570802F8570C80F8C2F837060
:1058A000C695C69593E0000F111F9A95E1F7C80FB2
:1058B000C8018C2BEC010E94F82A00C068E08C2FF4
:1058C0000E94562B90E19A95F1F752985A9A4A9B6A
:1058D00035C087E090E04A9933C0F801E35DFE4FA0
:1058E0006381611561F02091A4013091A50184814B
:1058F0009581820F931F0E942A2B811519F10E9416
:10590000F02A80E28A95F1F75A98529A90E19A9596
:10591000F1F7F801E35DFE4F6081611551F02091D0
:10592000A4013091A50181819281820F931F0E9471
:10593000792B0E94F82A789481E008C000C0C7CF74
:10594000019749F4529A5A9A789480E0DF91CF9166
:105950001F910F91089500C0BECF2F923F924F929A
:105960005F926F927F928F929F92AF92BF92CF92EF
:10597000DF92EF92FF920F931F93CF93DF93CDB7F8
:10598000DEB7CA1BDB0B0FB6F894DEBF0FBECDBF70
:1059900009942A88398848885F846E847D848C8441
:1059A0009B84AA84B984C884DF80EE80FD800C814A
:1059B0001B81AA81B981CE0FD11D0FB6F894DEBF2D
:1059C0000FBECDBFED010895991B79E004C0991F6A
:1059D000961708F0961B881F7A95C9F78095089549
:1059E00087FB082E062687FD819567FD61950E943D
:1059F000E42C0EF4919507FC81950895AA1BBB1B1E
:105A000051E107C0AA1FBB1FA617B70710F0A61BBE
:105A1000B70B881F991F5A95A9F780959095BC01DF
:105A2000CD01089597FB072E16F4009407D077FD5B
:105A300009D00E94FE2C07FC05D03EF4909581957C
:105A40009F4F0895709561957F4F0895EE0FFF1F4A
:105A50000590F491E02D09940E94B82E332312F49E
:105A60008A1B9B0B0C94362D0E94B82EB7FF08950D
:105A7000821B930B0895002E083090F0982F872FEB
:105A8000762F652F542F432F322F22270850F4CF23
:105A9000220F331F441F551F661F771F881F991F32
:105AA0000A95B2F7002D089597FD1094002E083046
:105AB00098F00850232F342F452F562F672F782F1B
:105AC000892F912DF4CF15949795879577956795A4
:105AD00057954795379527950A95AAF71124002DD4
:105AE0000895CF92DF92EF92FF92CF93DF93CDB7DD
:105AF000DEB72A970FB6F894DEBF0FBECDBF8987F9
:105B00009A87A985BA852D913D914D915C91298304
:105B10003A834B835C83232B242B252B41F424E2F3
:105B200039ED4BE557E029833A834B835C836981E8
:105B30007A818B819C812DE133EF41E050E00E941E
:105B4000642E69017A01A7EAB1E49B01AC010E94CD
:105B5000832E69837A838B839C83ACEEB4EFA70199
:105B600096010E94912E9B01AC0189819A81AB81A3
:105B7000BC81820F931FA41FB51FB7FF03C00197FD
:105B8000A109B048E985FA8580839183A283B38314
:105B90009F772A960FB6F894DEBF0FBECDBFDF9178
:105BA000CF91FF90EF90DF90CF9008950E94712DDC
:105BB000089580E091E00E94712D0895B0E0A0E08A
:105BC0008093000190930101A0930201B09303011F
:105BD0000895FC014150504030F001900616D1F775
:105BE0003197CF010895882799270895FB01DC019B
:105BF00004C08D910190801921F441505040C8F7A4
:105C0000881B990B0895FB01DC0102C001900D92E5
:105C100041505040D8F70895F999FECF92BD81BD0B
:105C2000F89A992780B50895A6E1B0E044E050E0E5
:105C30000C94562EA8E1B0E042E050E00C94562EB1
:105C4000DC01A40FB51F4150504048F0CB01840F38
:105C5000951F2E910E94312E41505040D0F708954B
:105C6000262FF999FECF92BD81BDF89A019700B415
:105C7000021639F01FBA20BD0FB6F894FA9AF99AB5
:105C80000FBE08950396272F0E94312E0E94302EBA
:105C9000252F0E94312E242F0C94312E0196272F70
:105CA0000E94312E0C94302EDC01CB01FC01F999BD
:105CB000FECF06C0F2BDE1BDF89A319600B40D9258
:105CC00041505040B8F70895052E97FB1EF40094FC
:105CD0000E947B2E57FD07D00E94962E07FC03D012
:105CE0004EF40C947B2E50954095309521953F4F66
:105CF0004F4F5F4F089590958095709561957F4FB8
:105D00008F4F9F4F08950E94B82EA59F900DB49F6E
:105D1000900DA49F800D911D11240895B7FF0C9440
:105D2000832E0E94832E821B930B0895A1E21A2ECC
:105D3000AA1BBB1BFD010DC0AA1FBB1FEE1FFF1F2F
:105D4000A217B307E407F50720F0A21BB30BE40B7F
:105D5000F50B661F771F881F991F1A9469F76095C6
:105D60007095809590959B01AC01BD01CF01089580
:105D7000A29FB001B39FC001A39F700D811D11248C
:105D8000911DB29F700D811D1124911D0895F894ED
:105D9000FFCF1B09230926092C09410941094109A3
:105DA000410941094109410941092F0934093809CB
:105DB0003E094F095509590977129E12A4129E12E5
:105DC000A412F7121913A4121714241478197C19A9
:105DD000A919AE19B219B419B619B8194B1B4F1B32
:105DE000411B471B531B571B5B1B4F1C791C801C03
:105DF000851C8A1C8F1C941C991C9E1CA31CA81C0F
:105E0000AD1CB01CB51CB81CBB1CBE1CC11CC41CEA
:105E10001B1BC71C5D1D5D1D961D961D531E701E10
:105E2000BD1DBD1D751EFF1E0E1F0E1FA21B0C1CCF
:105E3000AA1B741B781BAE1B7C1BB21BBE1B881BD2
:105E4000051C8C1BC21B901BC61BED1B941BCA1B85
:105E5000F41B9A1BD01BD81B801BB61B841BBA1BC0
:105E60009E1BD41BE41BFD1B031C6E1BA61B131CDB
:105E7000010000000101010201191A1B1C1D1E1F57
:105E8000202122003600363632363331F7F697C6F7
:105E9000343501EF09A20EB90EC00E669400000061
:105EA00001000000000000000401000000000000EC
:105EB00001050000000000000106000000040700CA
:105EC00000000000000B0B000000000000FF00BEFF
:105ED00000946697C63435000001020202020606ED
:105EE000060909090909090F0F0F0F0F0F151515DD
:105EF00018191919191919191919192323232323E1
:105F00002304000100FF0100010000FFFF00000169
:105F10000001FF000D04E200E900EA00B500B60050
:105F2000B700CD008301CC008A01920194012102C7
:105F3000230224022502260227022A02B300B4000B
:0C5F40006F0070009F01CB019F02A002C7
:00000001FF
